:020000040000FA
:040000006E303A28FC
:08000800A000030EA100831209
:1000100081018B100B11210E8300A00E200E090010
:0C007400203084008001840A6030040207
:10008000031C3C281230B000712183160C3085050A
:1000900087018312850187010730990000309A009B
:1000A000103083168E008312603083168F00831207
:1000B0000030831691008312C830831681008312AA
:1000C00031309000003083168C00831210308B008A
:1000D000831600309B001C141A088312BC00831680
:1000E00010309B001C141A088312BD008A21810164
:1000F0008E018F010B118B100B108C018B178F2031
:10010000311991205321B30B8D2803108519031445
:10011000B90DF03039020319AE21B6217F286400F1
:100120000800080031110130B7008B132030370769
:1001300083169B001C141A088312A4001030370782
:1001400083169B001C141A088312A3000030370783
:1001500083169B001C141A088312A2008B17321CF2
:10016000B72822090339A200A309A409A50901306F
:100170003702031DC0283D18C0283D143E147221CB
:1001800002303702031DC928BD18C928BD143E140A
:10019000752103303702031DD2283D19D2283D15A1
:1001A0003E14782104303702031DDB28BD19DB28FB
:1001B000BD153E147B2105303702031DE4283D1A8E
:1001C000E4283D163E147E2106303702031DED283B
:1001D000BD1AED28BD163E14812107303702031DDC
:1001E000F6283D1BF6283D173E14842108303702BF
:1001F000031DFF28BD1BFF28BD173E148721B70A2A
:10020000093037020318080095280130B600B30002
:10021000B400B500B70085018701B1138F20B30B7F
:100220002B29031085190314B90DF0303902031975
:100230004929B41F8501B41F8701B40B2B29370846
:10024000B6080319B60003192929FF308500870075
:10025000B6039630B400311D0E293111321C3529F8
:100260002D090339AD00AE09AF098B1320303707D4
:10027000BB002F08BA005C2110303707BB002E08E6
:10028000BA005C2100303707BB002D08BA005C21A2
:100290008B1785018701B70AB60109303702031CA5
:1002A0000E298A2108003E1C08003E101030BB00B9
:1002B0003D08BA005C2108008B133A0883161C1510
:1002C0009A0083123B0883169B0055309D00AA308C
:1002D0009D009C1464009C186A291C1183128B17C2
:1002E000080008000130BD0008000230BD00080011
:1002F0000430BD0008000830BD0008001030BD000B
:1003000008002030BD0008004030BD0008008030EB
:10031000BD00080001303D020319080002303D0213
:100320000319080004303D020319080008303D029B
:100330000319080010303D020319080020303D0267
:100340000319080040303D020319080080303D02C7
:10035000031908000130BD003E1408003E140310CC
:10036000BD0DBD1B3D14BD138A2108008F08031964
:1003700008008F0107303D050319AE2A02303D0504
:10038000031D51105408EB3C031805125118CB29DA
:10039000D40BD629D029D4035408C83C031CD62931
:1003A0000516F530D4005108013AD10002303D0560
:1003B000031DD1105508E63C03188512D118E32916
:1003C000D50BEE29E829D5035508B93C031CEE29C5
:1003D0008516F030D5005108023AD10002303D05B3
:1003E000031D51115608DC3C031805105119FB2957
:1003F000D60B062A002AD6035608B63C031C062A4A
:100400000514E630D6005108043AD10002303D050B
:10041000031DD1115708F03C03188510D119132A78
:10042000D70B1E2A182AD7035708D73C031C1E2AAD
:100430008514FA30D7005108083AD10002303D0542
:10044000031D51125808E03C03188710511A2B2A3B
:10045000D80B362A302AD8035808C13C031C362A48
:100460008714EA30D8005108103AD10006303D0513
:10047000031DD1125908D43C03180711D11A432A7D
:10048000D90B4E2A482AD9035908A73C031C4E2AE7
:100490000715DE30D9005108203AD10006303D055D
:1004A000031D51135A08BF3C03180710511B5B2A48
:1004B000DA0B662A602ADA035A089C3C031C662A77
:1004C0000714C930DA005108403AD10006303D0522
:1004D000031DD1135B08D73C03188712D11B732A65
:1004E000DB0B7E2A782ADB035B08BE3C031C7E2ADA
:1004F0008716E130DB005108803AD10006303D0517
:10050000031D52105C08F13C0318071252188B2A85
:10051000DC0B962A902ADC035C08CF3C031C962A4D
:100520000716FB30DC005208013AD20006303D05C8
:10053000031DD2105D08E93C03188711D218A32AC5
:10054000DD0BAE2AA82ADD035D08B23C031CAE2AEF
:100550008715F330DD005208023AD20018303D050D
:100560000319FE2ABD1DBA2A54083C3C031CBA2AB2
:1005700085018701D40B0800D0034630D4000B302E
:100580005002031DC42A05160A305002031DC92A51
:10059000851609305002031DCE2A0514083050027A
:1005A000031DD32A851407305002031DD82A87144F
:1005B00006305002031DDD2A071505305002031DC9
:1005C000E22A071404305002031DE72A871603307D
:1005D0005002031DEC2A071602305002031DF12AB7
:1005E000871501305002031DF52A12305002031CFA
:1005F0000800850187010C30D000080020303D053F
:100600000319482BD40B092B0508103A85008230BA
:10061000D400D50B102B0508203A85007D30D5007D
:10062000D60B172B0508013A85007330D600D70B7F
:100630001E2B0508023A85008730D700D80B252BE2
:100640000708023A87007730D800D90B2C2B07080F
:10065000043A87006B30D900DA0B332B0708013AD4
:1006600087005630DA00DB0B3A2B0708203A870068
:100670006E30DB00DC0B412B0708103A8700883016
:10068000DC00DD0B482B0708083A87008030DD00CE
:1006900040303D050319BF2B5408E63C03180512F2
:1006A000D40B6E2B0516F030D4002130DE07031872
:1006B0006C2BB130D507FA30D607C830D707643075
:1006C000D8079630D907BE30DA07AA30DB079A3050
:1006D000DC07C430DD076E2B8030BD005508823C3E
:1006E00003188512D50B772B85168C30D50056084C
:1006F000653C03180510D60B802B05146F30D6000F
:100700005708913C03188510D70B892B85149B3013
:10071000D7005808D73C03188710D80B922B8714A2
:10072000E130D8005908503C03180711D90B9B2B16
:1007300007155A30D9005A08873C03180710DA0BFE
:10074000A42B07149130DA005B08BD3C0318871214
:10075000DB0BAD2B8716C730DB005C08703C031841
:100760000712DC0BB62B07167A30DC005D08A73CBD
:1007700003188711DD0BBF2B8715B130DD008030EA
:0E0780003D050319C62B85018701DE01080027
:084000000B00030002000600A2
:02400E00CC33B1
:10420000FF00FF00FF00FF00FF00FF00FF00FF00B6
:10421000FF00FF00FF00FF00FF00FF00FF00FF00A6
:104220000100FF00FF00FF00FF00FF00FF00FF0094
:10423000FF00FF00FF00FF00FF00FF00FF00FF0086
:104240001000FF00FF00FF00FF00FF00FF00FF0065
:10425000FF00FF00FF00FF00FF00FF00FF00050060
:10426000FF00FF00FF00FF00FF00FF00FF00FF0056
:10427000FF00FF00FF00FF00FF00FF00FF00FF0046
:10428000FF00FF00FF00FF00FF00FF00FF00FF0036
:10429000FF00FF00FF00FF00FF00FF00FF00FF0026
:1042A000FF00FF00FF00FF00FF00FF00FF00FF0016
:1042B000FF00FF00FF00FF00FF00FF00FF00FF0006
:1042C000FF00FF00FF00FF00FF00FF00FF00FF00F6
:1042D000FF00FF00FF00FF00FF00FF00FF00FF00E6
:1042E000FF00FF00FF00FF00FF00FF00FF00FF00D6
:1042F000FF00FF00FF00FF00FF00FF00FF000000C5
:00000001FF
